:020000040000FA
:0400000013EF00F00A
:08000800006ED8CF02F0E0CF3A
:1000100001F0F2B2B3EC00F000D001C0E0FF0050FC
:1000200002C0D8FF1000806A816A826A0F0EC16E1A
:10003000070EB46E94909492949494969498949A93
:10004000949C949E9290929292949296929A939467
:100050009396939882908292829482968298829AC2
:10006000829C829E8090809280948096809A8194D7
:1000700081968198800E056E066E076E086E096E79
:100080000A6E0B6E0C6E0D6E0E6E0F6E106E116E94
:10009000126E136E146EAAEC00F0010E156E02ECD7
:1000A00001F0FF0E046E800E036E800EB16ED09EC6
:1000B000F28EF28C296A10EE05F020EE17F0100E89
:1000C000276EE6CFDEFF272EFCD7828082828284D5
:1000D00082868288828A828C828E808080828084DE
:1000E0008086808A818481868188286A174E8290E2
:1000F000184E8292194E82941A4E82961B4E829806
:100100001C4E829A1D4E829C1E4E829E1F4E8090D7
:10011000204E8092214E8094224E8096234E809ACB
:10012000244E8194254E8196264E81981550166E48
:10013000A4EC00F0A192B180A1A2FED7162EF8D7B0
:10014000282ED4D7B8D7B6D7B1900450B36E035089
:10015000B26E120093809382F18CF292F2882B6A35
:10016000080E2C6E1200B8EC00F0F292F288120029
:10017000D89081B2D88030322B502A6ED8902A364F
:10018000010ED8B0E828FA6E920E2A24D8B0FA2AC6
:10019000F96E02D00AD016D02C2E1200010E2B6E52
:1001A000060E2C6E30502D6E12002C2E1200020EF8
:1001B0002B6E080E2C6E30502E6ED8902E32D890AA
:1001C0002E3212002C2E1200000E2B6E080E2C6EFA
:1001D000200E2D62120030502F6E00EE05F02E50D2
:1001E0002FC0EBFF12000A0E316E010E336EC80EE7
:1001F000326E00000000322EFCD7332EF8D7312E9D
:10020000F4D712000A0E316EFA0E336EC80E326E3B
:1002100000000000322EFCD7332EF8D7312EF4D751
:1002200012000A0E316E336EC80E326E00000000EE
:10023000322EFCD7332EF8D7312EF5D712000A0E06
:10024000316E010E336E320E326E00000000322E1F
:10025000FCD7332EF8D7312EF4D7120002EC01F080
:0E02600002EC01F002EC01F002EC01F01200E1
:020000040030CA
:0E000000FF36FEFEFFFDFAFFFFFFFFFFFFFFD2
:00000001FF
